:1000000000308A001C28000021308400831300087F
:1000100003191B280130F800BF30F7006400F70B0C
:100020000E28F80B0C284A30F700F70B15280000B3
:100030006400800B0A280034840183131F30830579
:1000400083161F149F141F159F1107309C00FF304B
:100050008312A000831681131F149F141F159F1174
:1000600083121F108316091283129412A012200803
:1000700083168700831220162008831687008312B8
:10008000A0112008831687000130831294000030ED
:10009000831694000108C739083881008312900143
:1000A0000030F800920000308316920007309C0068
:1000B000050864000230F700F70B5C285F281C0875
:1000C00083120D1383169D018613831286138316E4
:1000D0000613831206138316861283128612831662
:1000E0000612831206128316061083120610831658
:1000F000861083128610831606118312061183164A
:100100008611831286110330A10004208316861302
:100110008312861383160613831206138316861220
:10012000831286168316061283120616831606108D
:10013000831206108316861083128610831606110A
:100140008312061583168611831286150430A100CA
:1001500004208316861383128613831606138312D4
:1001600006138316861283128612831606128312D2
:100170000612831606108312061083168610831249
:1001800086108316061183120615831686118312B4
:1001900086150230A1000420831686138312861769
:1001A0008316061383120613831686128312861291
:1001B0008316061283120612831606108312061087
:1001C0008316861083128614831606118312061571
:1001D00083168611831286150130A1000420831630
:1001E0008613831286178316061383120617831647
:1001F000861283128616831606128312061683163B
:100200000610831206148316861083128614831632
:100210000611831206158316861183128615033084
:10022000A1000420831686138312861383160613F7
:100230008312061383168612831286128316061201
:100240008312061283160610831206108316861078
:1002500083128610831606118312061183168611E7
:10026000831286110330A1000420831686138312A3
:1002700086178316061383120617831686128312B7
:10028000861683160612831206168316061083122C
:1002900006148316861083128614831606118312A1
:1002A000061583168611831286150330A1000420DB
:1002B000831686138312861383160613831206137E
:1002C0008316861283128612831606128312061272
:1002D0008316061083120610831686108312861466
:1002E000831606118312061583168611831286154E
:1002F0000130A1000420831686138312861383160F
:10030000061383120613831686128312861283162F
:100310000612831206128316061083120610831625
:100320008610831286108316061183120615831613
:100330008611831286150130A100042083168613CE
:1003400083128613831606138312061383168612EE
:100350008312861283160612831206128316061063
:1003600083120610831686108312861083160611D8
:100370008312061183168611831286150130A1009F
:10038000042083168613831286178316061383129E
:100390000617831686128312861683160612831298
:1003A000061683160610831206148316861083120F
:1003B0008610831606118312061183168611831286
:1003C00086110130A100042083168613831286173C
:1003D0008316061383120617831686128312861657
:1003E000831606128312061683160610831206144D
:1003F0008316861083128614831606118312061143
:1004000083168611831286110230A1000420831600
:100410008613831286178316061383120617831614
:100420008612831286168316061283120616831608
:100430000610831206148316861083128610831604
:10044000061183120611831686118312861101305C
:10045000A1000420831686138312861383160613C5
:1004600083120613831686128312861283160612CF
:100470008312061283160610831206108316861046
:1004800083128610831606118312061183168611B5
:10049000831286150130A10004208316861383126F
:1004A000861383160613831206138316861283128D
:1004B0008612831606128312061283160610831202
:1004C0000610831686108312861083160611831277
:1004D000061583168611831286150130A1000420AB
:1004E000831686138312861383160613831206134C
:1004F0008316861283128612831606128312061240
:100500008316061083120610831686108312861433
:10051000831606118312061583168611831286151B
:100520000130A100042083168613831286178316D8
:1005300006138312061783168612831286168316F5
:1005400006128312061683160610831206148316EB
:1005500086108312861483160611831206158316DD
:100560008611831286150330A1000420831686139A
:1005700083128617831606138312061783168612B4
:100580008312861283160612831206128316061031
:1005900083120610831686108312861083160611A6
:1005A0008312061583168611831286150130A10069
:1005B000042083168613831286178316061383126C
:1005C000061383168612831286128316061283126E
:1005D00006128316061083120610831686108312E5
:1005E0008610831606118312061183168611831254
:1005F00086150230A1000420831686138312861309
:100600008316061383120613831686128312861628
:10061000831606128312061683160610831206141A
:100620008316861083128614831606118312061110
:1006300083168611831286110130A10004208316CF
:1006400086138312861383160613831206178316E6
:1006500086128312861683160612831206168316D6
:1006600006108312061483168610831286148316CE
:100670000611831206158316861183128611023025
:10068000A100042083168613831286138316061393
:100690008312061383168612831286168316061299
:1006A000831206168316061083120614831686100C
:1006B000831286148316061183120611831686117F
:1006C000831286110130A100042083168613831241
:1006D0008617831606138312061383168612831257
:1006E00086128316061283120612831606108312D0
:1006F0000610831686108312861083160611831245
:10070000061183168611831286150230A10004207B
:100710008316861383128617831606138312061711
:10072000831686128312861283160612831206120D
:100730008316061083120610831686108312861005
:1007400083160611831206158316861183128615E9
:100750000130A100042083168613831286178316A6
:1007600006138312061783168612831286168316C3
:1007700006128312061683160610831206148316B9
:1007800086108312861483160611831206158316AB
:100790008611831286154530A10004208316861326
:1007A000831286138316061383120613831686128A
:1007B00083128612831606128312061283160610FF
:1007C0008312061083168610831286108316061174
:1007D0008312061183168611831286110330A1003D
:1007E000042083168613831286138316061383123E
:1007F0000613831686128312861683160612831238
:1008000006168316061083120610831686108312AE
:10081000861083160611831206158316861183121D
:1008200086150430A10004208316861383128613D4
:1008300083160613831206138316861283128612FA
:1008400083160612831206128316061083120610F0
:1008500083168610831286108316061183120615DE
:1008600083168611831286150230A1000420831698
:1008700086138312861783160613831206138316B4
:1008800086128312861283160612831206128316AC
:1008900006108312061083168610831286148316A0
:1008A00006118312061583168611831286150130F0
:1008B000A10004208316861383128617831606135D
:1008C0008312061783168612831286168316061263
:1008D00083120616831606108312061483168610DA
:1008E0008312861483160611831206158316861149
:1008F000831286150330A100042083168613831209
:100900008613831606138312061383168612831228
:10091000861283160612831206128316061083129D
:100920000610831686108312861083160611831212
:10093000061183168611831286110330A10004204C
:1009400083168613831286178316061383120617DF
:1009500083168612831286168316061283120616D3
:1009600083160610831206148316861083128614CB
:1009700083160611831206158316861183128615B7
:100980000330A10004208316861383128613831676
:100990000613831206138316861283128612831699
:1009A000061283120612831606108312061083168F
:1009B0008610831286148316061183120615831679
:1009C0008611831286150130A10004208316861338
:1009D0008312861383160613831206138316861258
:1009E00083128612831606128312061283160610CD
:1009F0008312061083168610831286108316061142
:100A00008312061583168611831286150130A10004
:100A1000042083168613831286138316061383120B
:100A20000613831686128312861283160612831209
:100A30000612831606108312061083168610831280
:100A400086108316061183120611831686118312EF
:100A500086150130A10004208316861383128617A1
:100A600083160613831206178316861283128616C0
:100A700083160612831206168316061083120614B6
:100A800083168610831286108316061183120611B0
:100A900083168611831286110130A100042083166B
:100AA000861383128617831606138312061783167E
:100AB0008612831286168316061283120616831672
:100AC000061083120614831686108312861483166A
:100AD00006118312061183168611831286110230C5
:100AE000A10004208316861383128617831606132B
:100AF0008312061783168612831286168316061231
:100B000083120616831606108312061483168610A7
:100B1000831286108316061183120611831686111E
:100B2000831286110130A1000420831686138312DC
:100B300086138316061383120613831686128312F6
:100B4000861283160612831206128316061083126B
:100B500006108316861083128610831606118312E0
:100B6000061183168611831286150130A100042018
:100B700083168613831286138316061383120613B5
:100B800083168612831286128316061283120612A9
:100B900083160610831206108316861083128610A1
:100BA0008316061183120615831686118312861585
:100BB0000130A10004208316861383128613831646
:100BC0000613831206138316861283128612831667
:100BD000061283120612831606108312061083165D
:100BE0008610831286148316061183120615831647
:100BF0008611831286150130A10004208316861306
:100C0000831286178316061383120617831686121D
:100C10008312861683160612831206168316061092
:100C20008312061483168610831286148316061107
:100C30008312061583168611831286150330A100D0
:100C400004208316861383128617831606138312D5
:100C500006178316861283128612831606128312D3
:100C6000061283160610831206108316861083124E
:100C700086108316061183120615831686118312B9
:100C800086150130A100042083168613831286176F
:100C90008316061383120613831686128312861296
:100CA000831606128312061283160610831206108C
:100CB000831686108312861083160611831206117E
:100CC00083168611831286150230A1000420831634
:100CD0008613831286138316061383120613831654
:100CE0008612831286168316061283120616831640
:100CF0000610831206148316861083128614831638
:100D00000611831206118316861183128611013093
:100D1000A1000420831686138312861383160613FC
:100D200083120617831686128312861683160612FE
:100D30008312061683160610831206148316861075
:100D400083128614831606118312061583168611E4
:100D5000831286110230A1000420831686138312A9
:100D600086138316061383120613831686128312C4
:100D70008616831606128312061683160610831231
:100D800006148316861083128614831606118312A6
:100D9000061183168611831286110130A1000420EA
:100DA000831686138312861783160613831206137F
:100DB0008316861283128612831606128312061277
:100DC000831606108312061083168610831286106F
:100DD0008316061183120611831686118312861557
:100DE0000230A1000420831686138312861783160F
:100DF0000613831206178316861283128612831631
:100E0000061283120612831606108312061083162A
:100E10008610831286108316061183120615831618
:100E20008611831286150130A100042083168613D3
:100E300083128617831606138312061783168612EB
:100E40008312861683160612831206168316061060
:100E500083120614831686108312861483160611D5
:100E60008312061583168611831286154530A1005C
:080E70000420831664286300CE
:02400E00393F38
:00000001FF
